:100000000029A01123080319A0150530A2002730EC
:10001000A900103017200330A900E8301720A901EB
:1000200064301720A9010A3017202C081E28A800C8
:100030002D08A5002C08A40097202408A400A203E2
:100040000319A011230803192828220203182F28B6
:100050002408031DA011A0192F28303E35280800C0
:100060000C1E302899000314FC28211930280800A0
:1000700083169B0083161C141A089B0AFC28A901EE
:10008000A800FF30A807031CA907031CFC280330A5
:10009000A500E4304D204128A501F63EA400A509A5
:1000A000031C5828FE300000A40703185328A40797
:1000B0000000A50F5228000024185E28241860288C
:1000C0000800B601B701B801B9012130AA0088289B
:1000D000B60DB70DB80DB90D2C0836022D08031C4E
:1000E0002D0F37022E08031C2E0F38022F08031C79
:1000F0002F0F3902031C8828B9002C08B6022D08DE
:10010000031C2D0FB7022E08031C2E0FB802031478
:10011000A40DA50DA60DA70DAA0B68283908AF00E0
:100120003808AE003708AD003608AC00FC28AD0139
:10013000AC011030B000250DAC0DAD0D2808AC029F
:100140002908031C290FAD020318AD282808AC07A5
:1001500029080318290FAD070310A40DA50DB00B36
:100160009B28240808002030B000B601B701B80170
:10017000B9010310241CCA282C08B6072D0803183F
:100180002D0FB7072E0803182E0FB8072F080318D6
:100190002F0FB907B90CB80CB70CB60CA70CA60CEE
:1001A000A50CA40CB00BB92808001030B300A501B1
:1001B000A401B10CB00C031CE3282808A4072908EB
:1001C0000318290FA507A50CA40CAD0CAC0CB30BA0
:1001D000D9282C080800A400A71BF0202408FC281C
:1001E000A409A509A609A709A40A0319A50A0319C0
:1001F000A60A0319A70A0800831383120313080031
:10020000830183160F3099002030980083128030CC
:100210009800A0010130900097014A3083168600B3
:10022000FD308500073083129F008A113B2A8E0122
:100230008F010530970083160C1183120C11831661
:100240000C1583128A110C1927298A0121291508F6
:10025000D2001608D300043097000C118A110C1933
:1002600033298A012E291508D4001608D500520812
:100270005402D8005308031C013E5502D900053032
:1002800097000C118A110C1947298A014229150877
:10029000D6001608D7000C1152085602DA0053088F
:1002A000031C013E5702DB0083160C1183129701D9
:1002B00059085B028A11031C9D298A11031D6529B7
:1002C00058085A028A11031C9D295D08D802031C94
:1002D000D9035C08DE001030DF005E08A4005F0870
:1002E000A500A601A7015808AC005908AD00AE0151
:1002F000AF018A01B3202708D0002608CF002508C7
:10030000CE002408CD005008A7004F08A6004E08D4
:10031000A5004D08A4005A08AC005B08AD00AE0172
:10032000AF018A0161202708D0002608CF002508E8
:10033000CE002408CD008A11A129D001CF01CE0121
:10034000CD014F0850048A11031DB32910304E020D
:100350008A11031CB8298A11031DB32901304D02EB
:100360008A11031CB829D001CF011030CE00CD0175
:100370008A11D01FBF29D001CF01CE01CD010800C5
:100380003A08A4003B08A500A601A701AF01AE01F1
:10039000AD012D30AC008A01B3202708C800260823
:1003A000C7002508C6002408C5004808A70047085C
:1003B000A6004608A5004508A400AF01AE01023022
:1003C000AD00AC018A0161202508C4002408C300E7
:1003D0004808A7004708A6004608A5004508A4004D
:1003E000AF01AE010230AD00AC018A0161203708D7
:1003F000CA003608C9004A08B1004908B000A9017E
:100400000A30A8008A01D520C9002D08CA004A0870
:10041000CB00CC010310CB0C4908A4004A08A5006E
:10042000A601A701AF01AE010230AD00AC018A0107
:1004300061203908C8003808C7003708C6003608E8
:10044000C500470848048A11031D2A2AC6088A11D4
:1004500003193A2A4B08093A4C048A11031D372A1A
:10046000C30A0319C40ACC01CB018A113A2ACB0A68
:100470000319CC0A080064308A013F200130D10002
:1004800000308A013820C20001308A013820DC00A7
:1004900002308A013820DD008A0117214E08BB0096
:1004A0004D08BA008A1186187E2A86163B08AD00D0
:1004B0003A08AC00AE01AF01003EBC00F030BD0018
:1004C0002D0803182D0FBD07FF30BE002E0803189E
:1004D0002E0FBE07FF30BF002F0803182F0FBF07D6
:1004E0003F08A7003E08A6003D08A5003C088A0179
:1004F000EB20BA002508BB008A117F2A86128A11D8
:100500000519962A06160830BB0710303B028A11DF
:10051000031C942A8A11031D922A01303A028A117F
:10052000031C942A1030BB028A11972A06128A11E2
:10053000061B682B8A1185191B2B8A01C021C20852
:100540008A11031DDC2A41308A0130205A308A0189
:10055000302049308A0130204D308A01302055301A
:100560008A01302054308A01302048308A013020FE
:1005700020308A0130203D308A01302020308A012D
:1005800030200430A100A3014408AD004308AC00B2
:100590008A0101202E308A013020A3014C08AD00D1
:1005A0004B08AC008A01012020308A0130200D3038
:1005B0008A0130208A11192B45308A0130204C30B5
:1005C0008A01302045308A01302056308A0130209F
:1005D00041308A01302054308A01302049308A016C
:1005E00030204F308A0130204E308A0130202030B8
:1005F0008A0130203D308A01302020308A013020AD
:100600000430A100A3014408AD004308AC008A01F6
:1006100001202E308A013020A3014C08AD004B0888
:10062000AC008A01012020308A0130200D308A017F
:1006300030208A11632BC2088A11031D432B01301D
:10064000D10041303A07B4003B080318013EB50021
:1006500051083407C00035080318013EC10041307D
:100660008A0130203A088A0130203B088A01302074
:1006700051088A01302040088A01302041088A014F
:1006800030208A11632B45303A07B4003B08031829
:10069000013EB50051083407C00035080318013E7B
:1006A000C10045308A0130203A088A0130203B08D9
:1006B0008A01302051088A01302040088A01302008
:1006C00041088A0130208A11061B682B8A01632B9E
:0E06D0008A014C2A63008A016A2B8A016D2B75
:02400E00223F4F
:0642000000000D000B00A0
:00000001FF
